:10000000A028AC00F839A400A40CA40C240C84078C
:100010007320AC0000059C282C08031C030100067B
:100020002C0580069C28A01123080319A015053073
:10003000A2002730A700103029200330A700E830A5
:100040002920A70164302920A7010A302920280887
:100050003028A6002908A5002808A400802024082C
:10006000A400A2030319A011230803193A282202AD
:10007000031841282408031DA011A0194128303E6F
:10008000472808000C1E4228990003149C282119B7
:100090004228080083169B0083161C141A089B0A2A
:1000A0009C28A701A600FF30A607031CA707031C76
:1000B0009C280330A500E5305F205328A501F63EBB
:1000C000A400A509031C6A28FE300000A407031839
:1000D0006528A4070000A50F6428000024187028D4
:1000E00024187228080000308A002C08073982077B
:1000F0000134023404340834103420344034803461
:10010000A901A8011030AA00250DA80DA90D2608E7
:10011000A8022708031C270FA902031896282608FF
:10012000A80727080318270FA9070310A40DA50D7A
:10013000AA0B842824089C28831383120313080025
:1001400083160F3099002030980083128030980079
:10015000A001423083168600FD30850007308312EF
:100160009F00012985100830A400A40BB5280800C1
:100170000830A400A40BBA2885140830A400A40BEE
:10018000BF28080064305E200130B7000430370219
:100190000318D0280610B820B220B70A031DC628BD
:1001A00064305E200614B820B22006100130B7007B
:1001B000053037020318E128B820B220B70A031D22
:1001C000D82808000A30B700303084003708003ED5
:1001D00001200310051803140C200930B700B820C3
:1001E000B22032305E20303084003708003E0120DB
:1001F0000310051803140C200130B7020318EF2870
:1002000008008615851006108612B22006160130E9
:10021000A700F43052200612BD01BC01BB01003022
:100220004A20BA00861585100610B101B0010130D0
:10023000A500F4305F208611C220E22086150F3021
:100240003D0203182A293008BB0731080318013E74
:10025000BC07BD0A8519632986163C08A5003B0822
:10026000A400A7013D08A6008020B0002508B10029
:10027000453042204C3042207230422061304220D2
:100280007730422064304220613042207430422076
:1002900061304220203042203D3042202030422038
:1002A0000430A100A3013108A9003008A8001320E0
:1002B0000D3042200A304220BD01BC01BB01861234
:1002C000C83051208F290130061B0301AF000130D7
:1002D00005190301AF0403198F29861641303B0726
:1002E000AD003C080318013EAE003D082D07B800E4
:1002F0002E080318013EB900413042203B0842203D
:100300003C0842203D08422038084220390842205B
:10031000BD01BC01BB018612061B8F298C29122945
:0603200063009029922900
:02400E00223F4F
:024200000000BC
:00000001FF
